:100000000C9478050C94E3050C9489090C94E30591
:100010000C94E3050C94E3050C94E3050C94E305C0
:100020000C94E3050C94E3050C942F180C94E30551
:100030000C9445260C94E3050C94E3050C94E3051D
:100040000C94E3050C94E3050C94E3050C94E30590
:100050000C94E3050C949A260C94E3050C94E305A8
:100060000C94E3050C94E3050C94E3050C94E30570
:100070000C94E3050C94E3050C94E3050C94E30560
:100080000C94E3050C94E3050C94E3050C94E30550
:100090000C94E3050C94E305590B5B0B670B670BA2
:1000A000670B670B670B670B5D0B5F0B610B670BD8
:1000B000670B5B0B690B670B670B230B590B670B0C
:1000C000670B5F0B670B670B670B670B670B670BA8
:1000D000610B590B450B670B490B670B670B670BE4
:1000E000250B5D0B670B670B530B670B670B670BE0
:1000F000270B650B670B470B670B5B0B670B670BDE
:10010000570B4B0B670B4D0B5F0B670B670B670BAD
:10011000550B4F0B670B670B670B670B670B670B79
:10012000670B510B670B290B670B670B5D0B670B9D
:10013000670B650B670B670B670B670B670B670B31
:10014000670B670B670B2B0B670B670B670B530B6F
:10015000670B670B670B670B670B670B670B670B0F
:10016000670B670B2D0B670B2F0B310B670B670BA7
:10017000670B330B350B370B670B390B3B0B670BDF
:10018000670B670B630B3D0B670B410B3F0B430B7F
:10019000670B670B670B670B650BC60BD40BE00B8C
:1001A000E00BB80BE00BE00BE00BE00BE00BE00B1F
:1001B000E00BE00BE00BE00BE00BE00BE00BBA0B0D
:1001C000E00BBC0BE00BE00BE00BE00BD80BE00B03
:1001D000EF0BD60BE00BE00BE00BE00BE00BE00BC2
:1001E000E00BE00BE00BE00BE00BE00BE00BB00BE7
:1001F000CC0BBE0BD00BE00BC00BE00BC40BE00B29
:10020000CE0BC20BD20BC80BCA0BE00BE00BE00B02
:10021000E00BE00BE00BE00BB20BB40BB60BDA0B10
:10022000DC0BE00BE00BE00BDE0BCF0CED0C000D5C
:100230001A0D280D340D540D6B0D8E0DAB0DB20E35
:10024000DE0E560FA30F7E0FC00FE80FF00FF60F54
:10025000FA0F001080108210841086108810901001
:10026000901090108A108C108E107A16A116991783
:10027000A1169917ED161017991767177617541CC2
:10028000541C8C1C8C1C071D1B1F1B1F1B1F3B1D84
:100290001B1FE31CE31CD51E1B1FEA1E081F007B4F
:1002A00046010203763A687F6577482B353B6978CB
:1002B000796439141E3C6A7A1D16041A1F3D6B06B8
:1002C0001B070821203E6C2C19091715223F6D11C0
:1002D000050B0A1C23406E7E100D182425416F3635
:1002E0000E0C122726427037380F33132D437175C9
:1002F00034322F2E44727C7D283031744573515036
:100300004A524D492A5466594F5C5F4C4B4E6263CA
:100310005A5D5E60295367585B565761475548429E
:10032000403E3C3A3B456843413F3D2B357E697A30
:10033000790078141E7C6A7B1D16041A1F7F6B06D9
:100340001B070821204D6C2C19091715224A6D1125
:10035000050B0A1C234C6E49100D182425516F36CD
:100360000E0C1227264F7037380F33132D5271752C
:1003700034502F2E4E72397D283065314B735464C2
:10038000586776012A773259745C5F6602036263AC
:100390005A5D5E60295344575B5655614746802934
:1003A0001E1F20212223242526272D2E2A2B141A16
:1003B0000815171C180C12132F302878041607097B
:1003C0000A0B0D0E0F33343579311D1B061905113B
:1003D000103637387D557A2C393A3B3C3D3E3F400C
:1003E00041424353475F6061565C5D5E57595A5BBB
:1003F00062634648324445677B7F65030102525081
:10040000514F68696A6B6C6D6E6F707172580049FC
:100410004C754A4D734B4E767C777E7466547225CC
:100420003032582000623A2530345820006525309B
:10043000325820002146554C4C21200021464621AF
:100440002000522000723A253034582000643A25AA
:10045000752000633A257520006973723A2530349F
:1004600058200077253032582000214353335F460F
:1004700030210A00214353335F5245414459210A38
:1004800000214353335F5245534554210A00214311
:1004900053325F45305F4630210A00214353325FBB
:1004A0004630210A00214353325F4530210A0021A2
:1004B0004353325F494E4954210A00214353315F6F
:1004C00045305F25303258210A000A5B4F56525D95
:1004D00020004C2575200053257520000A49443A18
:1004E0002530345828257325732920000A556E6B52
:1004F0006E6F776E2049443A205265706F72742097
:10050000746F20544D4B20004E4720004F4B20006D
:100510000A353537365F43533832683A004D6F75C8
:1005200073653A206E6F7420737570706F727465A6
:10053000640A00522575200057257520005725753F
:10054000200057257520005825752000412575206D
:100550000049257520005B4348475D20000A25754A
:10056000205052543A25303258204953523A2530BF
:10057000345820005B5253545D20000A25752045F5
:1005800052523A25303258204953523A2530345885
:1005900020000A4B6579626F617264207374617226
:1005A000742E0A000A55534220636F6E66696775A0
:1005B0007265642E0A000A0A544D4B3A3261303497
:1005C000373166642F4C5546410A0A00340349000E
:1005D00042004D0020005000430020006B006500E9
:1005E000790062006F006100720064002000630007
:1005F0006F006E0076006500720074006500720086
:1006000000000E0374002E006D002E006B002E0003
:1006100000000403090409027400040100A0320967
:100620000400000103010100092111010001224021
:10063000000705810308000A090401000103000006
:10064000000921110100012236000705820308007C
:100650000A0904020002030000000921110100013F
:100660002222000705830320000107050303200061
:100670000109040300010300000009211101000128
:100680002239000705840320000112011001000037
:100690000008EDFEEE1B0100010200010501090644
:1006A000A101050719E029E7150025019508750145
:1006B0008102050819012905950575019102950129
:1006C000750391010507190029F71500250195F813
:1006D00075018102C00631FF0974A1010975150079
:1006E00026FF009520750881020976150026FF0077
:1006F000952075089102C005010980A101850216A7
:1007000001002637001A81002AB700751095018173
:1007100000C0050C0901A1018503160100269C02F9
:100720001A01002A9C02751095018100C00501097B
:1007300006A101050719E029E715002501950875AF
:1007400001810295017508810105081901290595A6
:10075000057501910295017503910105071900299D
:10076000FF150026FF00950675088100C0636F6EB7
:1007700073756D65723A20253034580A00737973A9
:1007800074656D3A20253034580A000A002530324D
:100790005820006B6579626F6172643A20004C45A5
:1007A000443A20253032580A0025583A253038621C
:1007B00025730A000A202030313233343536370AA7
:1007C0000064656C5F6B65795F6269743A20636190
:1007D0006E27742064656C3A20253032580A006117
:1007E00064645F6B65795F6269743A2063616E2748
:1007F00074206164643A20253032580A003F004377
:100800003E20004C25640A000A092D20436F6E73B8
:100810006F6C65202D0A4553432F713A0971756934
:10082000740A000A092D204D61676963202D0A644E
:100830003A0964656275670A783A096465627567A2
:10084000206D61747269780A6B3A09646562756734
:10085000206B6579626F6172640A6D3A0964656242
:100860007567206D6F7573650A763A0976657273E0
:10087000696F6E0A733A097374617475730A633A27
:1008800009636F6E736F6C65206D6F64650A302D40
:10089000343A096C61796572302D34284631302D37
:1008A0004634290A506175733A09626F6F746C6F30
:1008B000616465720A6E3A094E4B524F0A003F005E
:1008C0004E4B524F3A206F66660A004E4B524F3ADB
:1008D000206F6E0A0074696D65725F7265616433C2
:1008E0003228293A202530346C580A006B65796229
:1008F0006F6172645F6E6B726F3A2025580A006BED
:100900006579626F6172645F69646C653A2025582D
:100910000A006B6579626F6172645F70726F746FE9
:10092000636F6C3A2025580A00686F73745F6B65BB
:1009300079626F6172645F6C65647328293A20255F
:10094000580A000A092D20537461747573202D0A0A
:10095000004743433A20352E342E30204156522D45
:100960004C4942433A20322E302E30204156525FBD
:10097000415243483A2061767235310A004F505453
:10098000494F4E533A204C55464120455854524108
:100990004B455920434F4E534F4C4520434F4D4DEF
:1009A000414E44204E4B524F204B45594D41505FD4
:1009B00053454354494F4E20424F4F544C4F4144AE
:1009C00045525F53495A450A004255494C443A2022
:1009D0003261303437316664202831323A30333A6C
:1009E0003437204A756E2020332032303231290AC4
:1009F000005649443A2030784645454428742E6DC7
:100A00002E6B2E29205049443A203078316265659A
:100A10002849424D205043206B6579626F617264B2
:100A200020636F6E76657274657229205645523A5E
:100A3000203078303030310A00444553433A206347
:100A40006F6E766572742049424D205043206B656D
:100A500079626F61726420746F205553420A000AF4
:100A6000092D2056657273696F6E202D0A000A6D7C
:100A70006F7573653A206F66660A000A6D6F75734D
:100A8000653A206F6E0A000A6B6579626F61726465
:100A90003A206F66660A000A6B6579626F6172645C
:100AA0003A206F6E0A000A6D61747269783A206F9D
:100AB00066660A000A6D61747269783A206F6E0A80
:100AC000000A64656275673A206F6E0A000A646501
:100AD0006275673A206F66660A000A0A626F6F7471
:100AE0006C6F616465722E2E2E2000433E20000044
:100AF00011241FBECFEFD0E2DEBFCDBF04B603FE90
:100B000049C08091AC039091AD03A091AE03B09128
:100B1000AF038730904BA740B04B09F03BC0109219
:100B2000AC031092AD031092AE031092AF0314BE4B
:100B30000FB6F894A895809160008861809360005A
:100B4000109260000FBE1092010810920008E3E0BE
:100B5000F0E089E080935700E491E695E370E1507E
:100B6000E33040F4F0E0EE0FFF1FEE5AFE4F20811D
:100B7000318102C020E030E280E090E0A2E0B0E00D
:100B8000821B930BA109B109B595A79597958795F8
:100B9000FC01099511E0A0E0B1E0E4E4F1E500E03A
:100BA0000BBF02C007900D92A835B107D9F723E01B
:100BB000A8E5B1E001C01D92AC3AB207E1F70E948E
:100BC00095130C94A0280C940000FF93EF93E091F0
:100BD0005801F0915901309709F00995EF91FF9173
:100BE0000895FC018591803011F0EFDFFBCF08956F
:100BF000FF27E0E230E247FF0CC0419597FF09C0B4
:100C0000EDE26095709580959095611D711D811D37
:100C1000911D27FF02C0219530E350E2AA27660FFD
:100C2000771F881F991FAA1FA41710F0A41B639594
:100C30005A95A9F7AA3008F0A95FA05DAF93F39584
:100C4000611571058105910541F7ED3211F4EF93BE
:100C5000F395F21718F43F93F395FBCF8F91B5DF1F
:100C6000FA95E1F70895E991F9918591803021F0A5
:100C7000853219F0AADFF9CF089520E0E894559164
:100C80005532C1F3503311F4689455915A3348F4F6
:100C9000505390F3220F022E220F220F200D250F0A
:100CA000F4CF0EF4219589919991533619F3533766
:100CB00029F1533559F1BC0188279927E8945C360E
:100CC00021F48991999168945591543639F446EFFD
:100CD0007EF077FF0DC08FEF9FEF0AC055374AE0D7
:100CE00039F0583540E121F0523642E009F00895DC
:100CF000FF93EF937DDFEF91FF91B7CFFF93EF93DA
:100D0000FC0181918030B9F360DFFBCFFF93EF935B
:100D100068DFF1CFDF93CF93CDB7DEB72596A3DFA2
:100D2000CF91DF910895282F80916501823071F075
:100D30008330B1F0813001F5E62FF0E038E0739FA9
:100D4000E00DF11D1124E256FC4F13C0E62FF0E038
:100D500088E0789FE00DF11D1124E25EFC4F09C090
:100D6000E62FF0E038E0739FE00DF11D1124E2560C
:100D7000FD4FE491E03819F480E090E008959E2F53
:100D80009077892F90E034E0959587953A95E1F733
:100D900038E0239F800D911D112444E0880F991F96
:100DA0004A95E1F7EF709C012E0F311DF901EE0F0E
:100DB000FF1FE050F8498591949108955998519AF0
:100DC00008955198599A08955898509A08955098AE
:100DD000589A08955198599A85E08A95F1F700003C
:100DE00089B18695817008955098589A85E08A95C2
:100DF000F1F7000089B181700895CF93DF93EC0182
:100E00000E94EA06882341F0209731F085E08A9518
:100E1000F1F700002197F4CFCE01DF91CF91089533
:100E2000CF93DF93EC010E94EA06811108C020975E
:100E300031F085E08A95F1F700002197F4CFCE01DB
:100E4000DF91CF9108952E9826982F9827980E9489
:100E5000DE060E94E706E9E6F0E080818860808394
:100E6000E9980895E19AE99A0E94E1060C94E70650
:100E7000E9980E94DE060C94E706CF93DF932FB724
:100E8000F894C0910201D0910301CE018827811509
:100E90009F4F19F080E09FEF02C08FEF90E08C2B06
:100EA0009D2B90930301809302012FBFCE019927C0
:100EB0008F3F910581F5CD2FDD27C03FD10551F042
:100EC000CF3FD10509F451C080919903C034D105B9
:100ED00099F407C08091990380FF33C08CE394E0BC
:100EE00004C080FF2EC084E394E09F938F930E9400
:100EF0008A060F900F9025C080FF37C0DF93CF93F5
:100F00008DE294E09F938F930E948A060F900F903A
:100F10000F900F902AC0CE018F6F019699F08091AB
:100F2000990380FF0CC0DF93CF9385E294E09F93F9
:100F30008F930E948A060F900F900F900F90CD2FE5
:100F400001C0CFEF8091990380FF0CC01F92CF9317
:100F50008EE194E09F938F930E948A060F900F90EA
:100F60000F900F908C2F90E002C08FEF9FEFDF91DA
:100F7000CF910895CF93CAE1C15069F00E943D0717
:100F80008F3F2FEF920749F48FE99FE00197F1F728
:100F900000C00000F1CF8FEF9FEFCF910895109226
:100FA0005E0110925D0110925C0110925B0180E085
:100FB00090E890930101809300018FEF9FEF909351
:100FC00003018093020108953F924F925F926F92C6
:100FD0007F928F929F92AF92BF92CF92DF92EF92C9
:100FE000FF920F931F93CF93DF93C82F10925B0153
:100FF0008091990380FF0CC01F92CF9383E694E009
:101000009F938F930E948A060F900F900F900F90DE
:10101000809100019091010181159048A1F080918B
:10102000990380FF10C080910001909101019F936E
:101030008F9389E594E09F938F930E948A060F9087
:101040000F900F900F9080910001909101018115F8
:101050009048C9F70E94EA06811114C08091990353
:1010600080FF10C088EE93E00E9410079F938F933B
:1010700083E594E09F938F930E948A060F900F90D0
:101080000F900F900E94F406811120C08091990367
:1010900080FF1CC008EE13E00E94F40681110AC014
:1010A0000115110539F085E08A95F1F7000001502E
:1010B0001109F2CF1F930F938DE494E09F938F93C8
:1010C0000E948A060F900F900F900F90E9988BE086
:1010D000E82EFF24F394D0E03324339496E0492E95
:1010E00027E0522E38E0B32E45E0A42E54E0952E92
:1010F00063E0862E72E0772E66246394E2E4CE2EBF
:10110000E4E0DE2E0E94DE060E94E7068FE193E017
:101110000197F1F700C000000E94E4068FE193E020
:101120000197F1F700C000000E94E10680E197E21C
:101130000E94FD06892B19F460925B01ADC000E0AE
:1011400010E090E59A95F1F7CE01002E02C095953A
:1011500087950A94E2F780FF04C0F3240E94E70613
:1011600002C00E94E40682E390E00E941007892BEF
:1011700019F470925B0190C082E390E00E94FD063A
:10118000892B19F480925B0187C00F5F1F4F0830D5
:101190001105B9F620E52A95F1F7FF2019F00E9414
:1011A000E70602C00E94E40682E390E00E94100776
:1011B000892B19F490925B016FC082E390E00E944A
:1011C000FD06892B19F4A0925B0166C080E58A9523
:1011D000F1F70E94E7060CE211E00E94F406882372
:1011E00051F00115110561F095E09A95F1F70000B5
:1011F00001501109F2CF012B19F00CE211E00CC0E3
:1012000040925B0149C00115110561F025E02A9566
:10121000F1F70000015011090E94F406882399F3A8
:10122000012B19F450925B0137C08CE291E00E94CF
:101230001007892B19F4B0925B012EC000910201B6
:10124000109103010E94CF070E94E1060E94E70669
:10125000E19AE99A0E94BA07D82FC92F0F3F8FEF62
:10126000180781F08091990380FF0CC01F930F93A2
:1012700085E494E09F938F930E948A060F900F90CD
:101280000F900F908FB7F894109303010093020111
:101290008FBF8D2F9C2F2BC080915B01813081F4FB
:1012A000EA94EE2069F010925B018091990380FF2F
:1012B00029CFDF92CF920E948A060F900F9022CF03
:1012C00080915B01806180935B010E94DE060E9439
:1012D000E7068FE39FE10197F1F700C000000E944D
:1012E000E1060E94E706E19AE99A8FEF9FEFDF910E
:1012F000CF911F910F91FF90EF90DF90CF90BF9013
:10130000AF909F908F907F906F905F904F903F90A5
:1013100008951F920F920FB60F9211242F933F93AF
:101320004F935F938F939F9329B180919A0340913C
:101330000001509101014115504819F480935A0160
:101340000FC090915A01891B833050F080910001A9
:101350009091010190935E0180935D0180E2DDC078
:1013600080910001909101019695879590930101DC
:101370008093000120FF09C080910001909101013C
:1013800090689093010180930001809100019091F9
:10139000010199278038910509F4F9C0A8F4803239
:1013A000910509F4F4C038F4009709F4F0C04097AF
:1013B00009F489C0A9C08034910509F4E8C08035DA
:1013C000910509F480C0A0C0803C910539F150F42A
:1013D0008039910509F477C0803A910509F094C0ED
:1013E00084E64DC0803D910509F46DC0803E9105B5
:1013F00009F08AC0809100019091010190935E01F3
:1014000080935D018091000190910101892F9927BE
:10141000909301018093000183E252C084E64999D0
:101420000FC0882369F095E09A95F1F7000081508C
:10143000F6CF882349F095E09A95F1F700008150A6
:101440004999F7CF8111A3C08091000190910101CA
:1014500090935E0180935D01809100019091010164
:10146000892F9927909301018093000182E228C07F
:10147000882379F095E09A95F1F700008150499B17
:10148000F7CF07C0882349F095E09A95F1F700005F
:1014900081504999F7CF81117AC0809100019091D4
:1014A000010190935E0180935D0180910001909114
:1014B0000101892F9927909301018093000181E216
:1014C00080935C0133C08091000190910101909361
:1014D0005E0180935D01809100019091010197FF71
:1014E00002C080E101C081E180935C018091000134
:1014F0009091010146E0969587954A95E1F7909382
:1015000001018093000112C08091000190910101BE
:1015100090935E0180935D0180E880935B018091F0
:101520005B0190E0982F88278F6F27C08091000182
:101530009091010199278F3F910511F480EFEDCF34
:10154000809103018F3F31F0809102018F3F11F0B4
:1015500080E4E3CF8091020190910301982F8827C6
:1015600090930301809302012091000130910101C9
:101570008091020190910301822B9093030180934B
:10158000020180E090E890930101809300019F9117
:101590008F915F914F913F912F910F900FBE0F90C0
:1015A0001F901895CF93C82F8DEE0E94E4078A3FB5
:1015B000910521F48C2FCF910C94E407CF910895DD
:1015C000E82FE695E695E695EF70F0E0E759FE4FD7
:1015D0004081282F277081E090E002C0880F991F7A
:1015E0002A95E2F7242F30E028233923232B11F406
:1015F000842B80830895E82FE695E695E695EF70B5
:10160000F0E0E759FE4F2081382F377081E090E0FD
:1016100002C0880F991F3A95E2F7422F50E0482305
:101620005923452B19F08095822380830895482FF4
:1016300050E0FA013397E138F10508F048C0E45B67
:10164000FF4F0C94972887E108958FE108958CE56A
:10165000089580E6089582E6089587E2089583E577
:1016600008958FE2089589E3089587E308958FE34D
:10167000089587E408958FE4089586E508958EE53A
:1016800008958FE7089580E0089585E608958EE631
:1016900008958FE6089580E3089588E3089580E42F
:1016A000089588E4089580E5089587E508958FE515
:1016B000089588E1089588E0089580E2089580E122
:1016C000089589E108958DE6089588E208958F7759
:1016D00008958FE008958B35D1F058F48131F9F0F9
:1016E00018F48E3081F00895833159F0843569F013
:1016F00008958D3571F068F0823669F08C3769F0A5
:10170000089581E1089584E508958BE508958DE5B8
:1017100008958AE608958EE0089587E708958FE09A
:1017200008958C3549F018F4833161F008958637B7
:1017300029F08E3729F0089581E508958EE7089500
:1017400086E708958DE50895CF93482F50E0FA017C
:101750007C97E834F105A0F5E353FF4F0C949728EC
:1017600085E53EC08AE53CC08BE53AC08CE538C0D3
:101770008DE536C08EE534C08FE532C080E630C0DE
:1017800081E62EC082E62CC083E62AC08FE628C000
:1017900081E726C082E724C084E722C085E720C015
:1017A00087E71EC088E71CC08AE71AC08CE718C00C
:1017B0008FE716C080E714C089E712C08BE710C01E
:1017C000C82F1F928F938BEB94E09F938F930E946F
:1017D0008A060F900F900F900F908C2F01C084E518
:1017E000CF9108950F931F93CF93DF930E94732699
:1017F0008C010E943D07EC01019631F4C8010E9462
:101800008B26843F9140A8F3CE01DF91CF911F91A9
:101810000F9108950E9423070C9432078091990339
:10182000816080939903E9E6F1E0119281E0E93764
:10183000F807D9F70895E82FF0E0E759FE4F8081C7
:101840000895E9E6F1E0119281E0E937F807D9F768
:101850000895982F80916501823048F092FB882787
:1018600080F990FD826091FD84600C94D20A089505
:101870001F93CF93DF9380915B018823B1F1C091D7
:101880005D01D0915E0110915B010E947326DF9390
:10189000CF931F921F939F938F938BE795E09F9316
:1018A0008F930E948A0680915B0180752DB73EB7A9
:1018B000285F3F4F0FB6F8943EBF0FBE2DBF81117A
:1018C0000EC0809164018B3051F484E795E09F93C2
:1018D0008F930E948A06109264010F900F901092CD
:1018E0005B0110925E0110925D0180915C01882382
:1018F00009F448C090915C0180916801981709F43F
:1019000041C0C0915D01D0915E0110915C010E94C7
:101910007326DF93CF931F921F939F938F938DE531
:1019200095E09F938F930E948A06809168012DB75E
:101930003EB7285F3F4F0FB6F8943EBF0FBE2DBF96
:1019400085FF04C090915C0194FD06C084FF12C025
:1019500080915C0185FF0EC0809164018B3051F451
:1019600086E595E09F938F930E948A06109264010A
:101970000F900F9080915C018093680110925E013E
:1019800010925D01E09164018E2F90E08C30910502
:1019900008F00AC4FC01EB5EFE4F0C9497280E94ED
:1019A00073269F938F9381E595E09F938F930E9479
:1019B0008A061092650110926701109266011092DA
:1019C00068010E94210C0E94041C0E9473269093BF
:1019D00063018093620181E060C00E943D0701962F
:1019E00019F082E08093640180916201909163011B
:1019F0000E948B26893B9B4008F4D6C382E015C029
:101A00000E9473269F938F938CE495E09F938F930E
:101A10000E948A068FEF0E94E4070F900F900F90AC
:101A20000F908A3F910521F486E080936401BCC346
:101A300083E0FBCF0E9438072E98269A2F98279A8A
:101A40000E947326909363018093620184E0EDCF3E
:101A500080916201909163010E948B26853F9140A5
:101A600008F4A2C385E0E1CF2E9826982F982798F6
:101A70000E94CF070E9432070E9473269F938F9384
:101A800087E495E09F938F930E948A060E947326B5
:101A9000909363018093620186E0809364010F90CC
:101AA0000F900F900F9080C30E943D07019609F49C
:101AB0007BC30E9473269F938F9382E495E09F934C
:101AC0008F930E948A060E947326909363018093ED
:101AD000620187E0E2CF80916201909163010E94F0
:101AE0008B26853F914018F089E0809364010E9425
:101AF0003D07019609F458C30E9473269F938F9364
:101B00008DE395E09F938F930E948A060E9473262F
:101B1000909363018093620188E0BFCF809162015E
:101B2000909163010E948B26853F914018F089E0D7
:101B3000809364010E943D07019609F435C30E9419
:101B400073269F938F9388E395E09F938F930E94D2
:101B50008A0689E0A2CF80915C018131C1F082EFD9
:101B60000E94E4078F3F3FEF9307A1F08A3F910562
:101B7000A1F40E94F20B8F3F2FEF920789F0D82F2C
:101B8000CC270E94F20B9E01282BC9010BC08DEFC0
:101B90009FEF08C08FEF9FEF05C08EEF9FEF02C051
:101BA00080E090E090936701809366010E94732625
:101BB0009F938F9383E395E09F938F930E948A0670
:101BC00080916601909167010F900F900F900F9098
:101BD000009711F482E031C08F3F3FEF930711F47B
:101BE00081E02BC09C012D5F3F4F2230310590F3E7
:101BF0008F3F910559F48DE195E09F938F930E945B
:101C00008A06109265010F900F9068C09C012558BC
:101C10003B4A2230310520F082392BEA920781F4C9
:101C200080EF0E94E4078A3F9105A1F683E00E94BD
:101C3000E4078A3F910571F683E0809365014EC009
:101C40009C0120593B4A2230310500F580E195E0A6
:101C50009F938F930E948A0680EF0E94E4070F9063
:101C60000F908A3F910549F482E80E94E4078A3F79
:101C7000910519F48CE095E002C088E095E09F930F
:101C80008F930E948A060F900F90A4CF803B3FEB6A
:101C9000930791F2882781152BEA920709F49ACFCE
:101CA00081153FEB930741F281159F4729F28CEE96
:101CB00094E09F938F930E948A0680EF0E94E4072E
:101CC0000F900F908A3F910509F0AACF82E00E9401
:101CD000E4078A3F910509F0A3CF7CCF809166018C
:101CE000909167018E3F3FEF930749F08D3F2FEFB3
:101CF000920741F0009749F04DE151E008C04EE1F4
:101D000051E005C048E151E002C044E251E02091B9
:101D10006501213039F0223041F0233049F020E3D1
:101D200031E008C02DE231E005C02AE231E002C016
:101D300025E331E05F934F933F932F939F938F93CE
:101D40008CED94E09F938F930E948A068AE08093A3
:101D500064018DB79EB708960FB6F8949EBF0FBE6C
:101D60008DBF22C20E9473269F938F9387ED94E0CC
:101D70009F938F930E948A060F900F900F900F9061
:101D800080916501823029F0833039F488EF0E9418
:101D9000E4070E9421190E94290C8BE080936401C2
:101DA0000E9473269F938F9382ED94E09F938F936D
:101DB0000E948A060F900F900F900F900E943D078F
:101DC000282F482F592F4F3F9FEF590709F4ECC197
:101DD0004115510519F04F3F510539F40E94210C6E
:101DE0000E94041C8AEC94E0A2C1809165018230BB
:101DF00009F44EC0833009F40BC1813009F0D4C11D
:101E000080916101823061F128F4882341F08130B2
:101E100099F03BC0833071F1843091F136C0203E9F
:101E200021F0213E21F482E022C081E020C0822FF7
:101E300027FF48C18F7776C1263339F118F42A324B
:101E400029F423C02A3A09F1263BF9F0822F27FD15
:101E500003C00E94A40B11C08F770E94A40B13C073
:101E60002D3121F02D3989F484E001C083E0809385
:101E700061019AC1253449F485E50E94E00A05C054
:101E8000253C19F485E50E94FB0A109261018CC182
:101E9000822FE09160014E2F50E04930510508F04B
:101EA000B4C0FA01EF5DFE4F0C9497284091660193
:101EB0005091670140595B4A4230510518F4822F16
:101EC0000E946B0B803E69F030F4833871F08438E7
:101ED00071F48FE788C0813E31F0803F41F481E0AA
:101EE0008CC082E08AC084E088C082E07CC087FF2A
:101EF000E9C00E94210C8FEA94E061C04091660124
:101F00005091670140595B4A4230510528F4213114
:101F100009F446C1213451F0293509F476C0203F37
:101F200019F0223121F471C083E067C08CE7109270
:101F3000600187FD03C00E94170BC4C00E94210CE2
:101F400085EA94E03CC04091660150916701405998
:101F50005B4A4230510518F4822F0E946B0B833884
:101F600021F0843821F48FE74EC082E04CC01092FB
:101F7000600187FFD7C00E94210C8BE994E01FC04D
:101F8000409166015091670140595B4A42305105CA
:101F900028F4213109F406C1213429F02231A9F1B4
:101FA000293511F432C08CE71092600187FD03C01F
:101FB0000E94170BB7C00E94210C8EE894E09F93FB
:101FC0008F930E948A060F900F9010926401ECC0CC
:101FD000243121F0203FC9F486E00FC085E00DC018
:101FE000273799F480E00E94E00A0FC0243169F499
:101FF00087E003C0203F49F488E080936001D4C0AB
:10200000273719F480E00E94FB0A10926001CCC0CF
:10201000822F2F3B41F028F496E5920F923070F416
:1020200002C02C3F59F410925F0181E894E09F9325
:102030008F930E948A06109264017DC090915F0187
:10204000913009F445C038F0923009F477C09330EC
:1020500009F493C0A9C040916601509167014239CB
:102060005B4A19F4822F0E94910B863809F168F4BB
:102070008338D1F020F4803819F582E076C08438B6
:10208000A9F08538E9F488E61DC08C38A9F030F451
:10209000873881F08B38A1F481E014C08D3871F05D
:1020A000803F71F481E061C082E00CC08FE70AC01C
:1020B00088E708C080E006C089E004C08AE002C06A
:1020C00087FD03C00E94E00A6FC084E794E02FC040
:1020D00010925F01409166015091670142395B4A5D
:1020E00019F4822F0E94910B482F50E0FA01E35817
:1020F000F109EB30F105A0F4E65DFE4F0C94972852
:1021000082E010C08FE70EC088E60CC088E70AC0E6
:1021100080E008C081E006C089E004C08AE002C017
:1021200087FD03C00E94FB0A3FC08AE694E09F93AC
:102130008F930E948A060F900F9036C0253279F057
:1021400030F4263171F02E3199F480E00BC0263244
:1021500021F0203F69F483E008C08DE503C083E5EA
:1021600001C081E50E94E00A05C080935F011CC0A8
:102170000E94210C10925F0117C02E3169F020F4EB
:102180002631B1F781E509C0253221F0263281F7E9
:102190008DE503C083E501C080E00E94FB0AEACF21
:1021A00083E1C5CE83E100CF81E0DF91CF911F9124
:1021B000089580919D0208950895CF93DF9300D0F4
:1021C0001F92CDB7DEB72091A303243021F523E081
:1021D00029839B838A8382E08093E9008FEF90912B
:1021E000E800815095FD06C095ED9A95F1F7000045
:1021F0008111F5CF8091E80085FF0DC040E050E0EF
:1022000063E070E0CE0101960E9449158091E800DC
:102210008E778093E8000F900F900F90DF91CF9111
:102220000895CF93DF9300D01F92CDB7DEB72091F2
:10223000A303243029F522E02983805891099B8348
:102240008A832093E9008FEF9091E800815095FDFB
:1022500006C095ED9A95F1F700008111F5CF8091B8
:10226000E80085FF0DC040E050E063E070E0CE0183
:1022700001960E9449158091E8008E778093E800CE
:102280000F900F900F90DF91CF910895CF93DF9330
:10229000EC019091A303943009F048C0809114019F
:1022A0008823D9F0809115018823B9F09093E90033
:1022B00081E8815049F09091E80095FD05C09AE2CF
:1022C0009A95F1F700C0F5CF8091E80085FF2EC008
:1022D00040E050E060E270E019C081E08093E900E6
:1022E00081E8815059F09091E80095FD07C0EFE337
:1022F000F1E03197F1F700C00000F3CF8091E800E2
:1023000085FF14C040E050E068E070E0CE010E941C
:1023100049158091E8008E778093E80080E2FE0105
:10232000ADE7B2E001900D928A95E1F7DF91CF9190
:102330000895CF93C0917B01C1110BC00E947F26ED
:10234000643C79408105910520F081E080937B0118
:10235000C1E08C2FCF910895FF920F931F93CF93DD
:10236000DF93D82F0FB607FE83C08091A30384307C
:1023700081F08091070190E001962091090130E001
:10238000822393232091080130E08217930709F0FC
:10239000CBC00E949911811110C08091070190E07B
:1023A00001962091090130E08223932320910801B6
:1023B00030E08217930709F0B7C00E9473268C01A2
:1023C000C091E900CF709091EC00892F817090FD51
:1023D00080E8C82B83E08093E90085E0F82E8091A7
:1023E000EB0085FD42C08091EB0080FF3EC08091F4
:1023F000EE0087FF3AC0809108019091070198177D
:1024000009F457C09091E80095FF8CC0E091050158
:10241000F0910601E80FF11D20818F5F9091090175
:102420008923809308012093F1008091E80085FDC5
:10243000E2CF8091E80080FFDECF8091E8008E77C8
:102440008093E800F0920401D6CF8091070190E0DC
:1024500001962091090130E0822393232091080105
:1024600030E08217930709F44AC0CF70C093E900A7
:1024700040910701842F90E001962091090130E0FE
:10248000822393232091080130E08217930709F4F7
:102490004EC0E0910501F0910601E40FF11DD083DB
:1024A000809107018F5F9091090189238093070133
:1024B0003EC08091E80085FF35C0D093F10081E0F7
:1024C0002091F2003091F300232B91F09091E800DD
:1024D00090FF0EC09091E80095FF03C01092F100AC
:1024E000F9CF9091E8009E779093E800F092040174
:1024F000882309F4AACFCF70C093E90018C0809157
:102500000401882309F4B1CF0E9473269C0180172F
:10251000910711F4890163CF909104019150909338
:102520000401F8CF80E0CCCF40910701B2CF80E02A
:10253000DF91CF911F910F91FF9008958091A20399
:10254000811104C00E94B1170C94131808951092C1
:10255000A2030895089542E061EC81E00E94C21454
:1025600042E061EC82E00E94C21442E261EC83E04E
:102570000E94C21442E261EC84E00C94C214809187
:10258000A503833009F455C030F4813071F08230F6
:1025900009F48EC008958A3009F47AC08B3009F4AA
:1025A00060C0893009F09CC020C08091A403813AAA
:1025B00009F096C08091E800877F8093E8008091C1
:1025C000A8039091A903892B21F460E28DE792E0A2
:1025D00003C060E080E090E070E00E94961580917A
:1025E000E8008B778093E80008958091A4038132FE
:1025F00009F076C08091A8039091A903009719F083
:10260000039709F06DC08091E800877F8093E80010
:102610008091E80082FD05C08091A3038111F8CF6D
:102620005FC08091F10080939D028091E8008B77DC
:1026300053C08091A403813A09F052C08091A8034D
:102640009091A903892B09F04BC08091E800877F06
:102650008093E8008091E80080FFFCCF8091140116
:1026600036C08091A4038132D9F58091A80390915E
:10267000A903892BA9F58091E800877F8093E80062
:102680000E94F7148091A603809314010C94041CFB
:102690008091A403813221F58091E800877F8093A7
:1026A000E8000E94F7148091A70380939E0208958A
:1026B0008091A403813AA1F48091E800877F809300
:1026C000E8008091E80080FFFCCF80919E0280931B
:1026D000F1008091E8008E778093E8000C94F71465
:1026E000089580919D0280937C0110929D020E942A
:1026F000210C0C94041C0C9471130E9420268091D0
:10270000A103882329F00E942D2681110C94AC147A
:1027100008950E94412680917C0180939D02089536
:102720000C94891308950C949213CF9384B7877FE8
:1027300084BF0FB6F894A89580916000886180935B
:102740006000109260000FBE90E080E80FB6F89431
:1027500080936100909361000FBE8CEA91E10E942A
:10276000F3258AE091E00E941C1986EB95E00E9417
:10277000F1050E940A0C0E94D0190E94B1170E9414
:10278000131878940E94D2198091A303843029F001
:102790000E9401190E949213F7CF84EA95E00E94EB
:1027A000F1050E94931382E995E00E94F105C3E0D0
:1027B0008091A303853019F40E947D13F9CF0E9404
:1027C000D6192091E4003091E50080917901909133
:1027D0007A012817390709F466C08091E4009091C6
:1027E000E50090937A01809379010E9499118823E2
:1027F00009F459C08091A303843009F054C080913A
:10280000E9008F702091EC00922F917020FD90E8EC
:10281000892BC093E9009091EB0090FF41C090910B
:10282000EE0097FF3DC09091080120910701291704
:1028300009F12091E80025FF1DC0E0910501F0910C
:102840000601E90FF11D30819F5F2091090192235C
:10285000909308013093F1009091E80095FDE3CF4B
:102860009091E80090FFDFCF9091E8009E779093E1
:10287000E800D9CF2091F2003091F300232B81F0B2
:102880009091E80090FF0CC09091E80095FF03C084
:102890001092F100F9CF9091E8009E779093E800B4
:1028A0008F708093E9000E94011982CF292F33276E
:1028B00023303105C9F060F42130310581F0223038
:1028C000310509F041C084E790E026E136E040C0E0
:1028D00021323105E1F02232310531F135C082E19A
:1028E00090E02AE836E034C099278130910549F01C
:1028F00028F0029749F5ECECF5E005C0E2E1F6E0DE
:1029000002C0E2E0F6E0849190E09F0121C06430D3
:102910007105D0F4660F771FFB01E65BFE4F208147
:10292000318189E090E014C06430710568F4FB01E6
:10293000EE0FFF1FEE5BFE4F20813181FB01E25C59
:10294000FE4F808190E004C080E090E020E030E025
:10295000FA0131832083089584E189BD86E189BD30
:1029600009B400FEFDCF8091D8008F7D8093D80000
:102970008091E00082608093E0008091E00081FD22
:10298000FCCF0895982F973068F59093E900981739
:1029900039F07091EC002091ED005091F00003C0EF
:1029A000242F762F50E021FD02C09F5FECCF3091A5
:1029B000EB003E7F3093EB003091ED003D7F309394
:1029C000ED003091EB0031603093EB007093EC0040
:1029D0002093ED005093F0002091EE0027FDE5CF0D
:1029E00080E008958F708093E90081E008958091E0
:1029F000A40387FF11C08091E80082FD05C080918B
:102A0000A3038111F8CF11C08091E8008B770BC030
:102A10008091A303882349F08091E80080FFF8CFDC
:102A20008091E8008E778093E80008952091E4007B
:102A30003091E50095E64091EC00842F817040FFD5
:102A400023C08091E80080FD1DC08091A3038823EE
:102A500099F0853099F08091EB0085FD11C040918F
:102A6000E4005091E5002417350729F3915011F047
:102A70009A01E1CF84E0089582E0089583E008950B
:102A800081E0089580E008954091E80042FFDDCFA5
:102A90000895CF92DF92EF92FF920F931F93CF93FF
:102AA000DF93EC018B017A010E941615811135C06C
:102AB000E114F10439F0F70180819181081B190BB1
:102AC000C80FD91FC12CD12C0115110529F18091F6
:102AD000E80085FD18C08091E8008E778093E800BB
:102AE0000E940119E114F10449F0F70180819181FC
:102AF000C80ED91ED182C08285E00FC00E94161573
:102B0000882311F30AC089918093F10001501109C3
:102B1000FFEFCF1ADF0AD8CF80E0DF91CF911F916E
:102B20000F91FF90EF90DF90CF9008952091AA032E
:102B30003091AB032617370748F06115710539F45A
:102B40002091E8002E772093E80001C0B901FC0134
:102B500020E06115710569F18091A3038823E1F1FB
:102B60008530E1F18091E80083FD3AC08091E80072
:102B700082FD2CC08091E80080FFEBCF8091F200B5
:102B80009091F3006115710551F08830910538F48A
:102B900021912093F100615071090196F3CF21E05A
:102BA000089709F020E08091E8008E778093E80094
:102BB000D0CF2111D1CF0AC08091A303882361F027
:102BC000853061F08091E80083FD0AC08091E800C3
:102BD00082FFF2CF80E0089582E0089583E00895B7
:102BE00081E008952091AA033091AB03261737079F
:102BF00048F06115710539F42091E8002E77209393
:102C0000E80001C0B901FC0120E06115710581F106
:102C10008091A303882309F43EC0853009F43DC0A8
:102C20008091E80083FD3BC08091E80082FD2DC0CB
:102C30008091E80080FFE9CF8091F2009091F3004D
:102C40006115710559F08830910540F42491209365
:102C5000F1003196615071090196F2CF21E0089799
:102C600009F020E08091E8008E778093E800CDCFD6
:102C70002111CECF0AC08091A303882361F0853053
:102C800061F08091E80083FD0AC08091E80082FF36
:102C9000F2CF80E0089582E0089583E0089581E016
:102CA00008951F93CF93DF93CDB7DEB7AA970FB6E2
:102CB000F894DEBF0FBECDBFE4EAF3E08091F100EF
:102CC000819323E0EC3AF207C9F70E94BF1280918A
:102CD000E80083FF2EC18091A4039091A503492FA2
:102CE00050E04A30510508F024C1FA01EB5CFE4F78
:102CF0000C949728803821F0823809F01AC108C056
:102D00008091A0039091A103992389F082600FC064
:102D10008091A8038F70873008F00BC18093E90081
:102D20008091EB0085FB882780F91092E900909153
:102D3000E800977F9093E8008093F1001092F100F3
:102D4000D1C0282F2D7F09F0F4C0882319F08230DC
:102D500061F0EFC08091A603813009F0EAC09330A2
:102D600009F080E08093A1032EC08091A603811119
:102D70002AC08091A8038F702FEF280F263008F00B
:102D8000D8C08093E9002091EB0020FF1CC0933055
:102D900021F48091EB00806214C09091EB0090616F
:102DA0009093EB0021E030E0A90102C0440F551FD1
:102DB0008A95E2F74093EA001092EA008091EB00D6
:102DC00088608093EB001092E9008091E800877F93
:102DD0008093E8000E94F714ACC08111AAC0109142
:102DE000A6031F778091E3008078812B8093E30016
:102DF0008091E800877F8093E8000E94F71480911B
:102E0000E80080FFFCCF8091E30080688093E300BE
:102E1000111102C082E001C083E08093A30389C046
:102E20008058823008F085C08091A6039091A70356
:102E30008C3D53E0950779F583E08A838AE28983A4
:102E40004FB7F894DE01139620E03EE051E2E32F05
:102E5000F0E050935700E49120FF03C0E295EF703B
:102E60003F5FEF708E2F90E0EA3010F0C79601C000
:102E7000C0968D939D932F5F243149F74FBF80916A
:102E8000E800877F8093E8006AE270E0CE01019657
:102E90000E94961516C06091A8037091A903AE0117
:102EA0004F5F5F4F0E945614BC01892B09F441C04B
:102EB0009091E800977F9093E80089819A810E9421
:102EC000F2158091E8008B778093E80032C080385B
:102ED00081F58091E800877F8093E80080919F03CF
:102EE0008093F1008091E8008E7772CF811121C02C
:102EF0008091A6039091A70399270297D4F480911B
:102F0000E800877F8093E8008091A60380939F0369
:102F10000E94F71480919F03811106C08091E30005
:102F200087FD02C081E001C084E08093A3030E947A
:102F3000AB128091E80083FF0AC08091E800877F90
:102F40008093E8008091EB0080628093EB00AA966A
:102F50000FB6F894DEBF0FBECDBFDF91CF911F91AA
:102F600008950E9422180E942A18E0EEF0E0808165
:102F700081608083E8EDF0E080818F77808319BCE9
:102F8000A7EDB0E08C918E7F8C9380818F7E8083C3
:102F90001092A20308950F931F93CF93DF930E9483
:102FA00022180E942A18C8EDD0E088818F77888384
:102FB00088818068888388818F7D8883E7EDF0E051
:102FC00080818068808319BC1092A30310929F03B4
:102FD0001092A1031092A00300EE10E0F80180818E
:102FE0008B7F808388818160888342E060E080E01D
:102FF0000E94C214E1EEF0E080818E7F8083E2EED9
:10300000F0E0808181608083808188608083F80126
:1030100080818E7F8083888180618883DF91CF91DA
:103020001F910F910895E8EDF0E080818F7E8083FD
:10303000E7EDF0E080818160808381E08093A203EE
:103040000C94CB17E8EDF0E080818C7F80831092A8
:10305000E20008951092DA001092E10008951F92A4
:103060000F920FB60F9211240BB60F922F933F932E
:103070004F935F936F937F938F939F93AF93BF9380
:10308000EF93FF938091E10082FF0BC08091E200FB
:1030900082FF07C08091E1008B7F8093E1000E9456
:1030A00000198091DA0080FF1FC08091D80080FF56
:1030B0001BC08091DA008E7F8093DA008091D90066
:1030C00080FF0DC084E189BD86E189BD09B400FEA1
:1030D000FDCF81E08093A3030E949E1205C019BC1E
:1030E0001092A3030E94A7128091E10080FF19C0F3
:1030F0008091E20080FF15C08091E2008E7F809376
:10310000E2008091E20080618093E2008091D8002B
:1031100080628093D80019BC85E08093A3030E944D
:103120007B138091E10084FF30C08091E20084FF36
:103130002CC084E189BD86E189BD09B400FEFDCFC4
:103140008091D8008F7D8093D8008091E1008F7EA0
:103150008093E1008091E2008F7E8093E200809175
:10316000E20081608093E20080919F03882311F048
:1031700084E007C08091E30087FD02C081E001C0C8
:1031800083E08093A3030E9490138091E10083FF6A
:1031900024C08091E20083FF20C08091E100877FFE
:1031A0008093E10082E08093A30310929F038091BB
:1031B000E1008E7F8093E1008091E2008E7F80931A
:1031C000E2008091E20080618093E20042E060E0F2
:1031D00080E00E94C2140E94AA12FF91EF91BF9159
:1031E000AF919F918F917F916F915F914F913F919F
:1031F0002F910F900BBE0F900FBE0F901F90189540
:103200000895CF938091A3038823A1F0C091E90092
:10321000CF709091EC00892F817090FD80E8C82BD1
:103220001092E9008091E80083FD0E945116CF7052
:10323000C093E900CF9108959093A4028093A302D4
:103240000895E091A302F091A402309721F001903B
:10325000F081E02D099480E00895EF92FF920F93A2
:103260001F93CF93DF93E091A302F091A4023097D4
:10327000B1F18C010280F381E02D099580919903D1
:1032800082FF2DC080FF04C083E997E00E94F10512
:10329000E80110E28DE8E82E87E0F82E809199038E
:1032A00080FF0BC088811F928F93FF92EF920E9444
:1032B0008A060F900F900F900F90115021961111C8
:1032C000EDCF8091990380FF0AC08BE897E0DF91F2
:1032D000CF911F910F91FF90EF900C94F105DF912A
:1032E000CF911F910F91FF90EF900895CF93DF93AF
:1032F0002091A1023091A2022817390709F1909379
:10330000A2028093A102E091A302F091A40230975F
:10331000B9F0EC010680F781E02D099580919903C1
:1033200082FF0EC080FF0CC0DF93CF938DE797E044
:103330009F938F930E948A060F900F900F900F908B
:10334000DF91CF910895CF93DF9320919F02309129
:10335000A0022817390709F19093A00280939F02D9
:10336000E091A302F091A4023097B9F0EC0100843F
:10337000F185E02D09958091990382FF0EC080FFB1
:103380000CC0DF93CF938DE697E09F938F930E94BD
:103390008A060F900F900F900F90DF91CF910895B4
:1033A0000C94791A0E946A260C940E0CBF92CF924C
:1033B000DF92EF92FF920F931F93CF93DF9300D092
:1033C00000D01F92CDB7DEB70E94380C06EA12E09B
:1033D000F12C8F2D0E941B0CB82EF801C080C8263E
:1033E00039F4F3940F5F1F4FF0E1FF12F2CF30C0BA
:1033F0008091990381FD0E947A1AD12CEE24E394E6
:103400008C2D8E21F9F0D982FA8291E08B2D8E21BC
:1034100009F490E09B830E9473268160782F9D833E
:103420008C8349815A816B818D810E94B01A4981B8
:103430005A816B817C818D810E940B26F8018081ED
:103440008E258083D394EE0CF8E0DF12D9CFC9CF5C
:103450008FEF89838A831B820E9473268160782F75
:103460009D838C8349815A816B818D810E94B01A22
:103470000E940A260E9421199091A502891741F104
:103480000E9421198093A5029091990392FF0EC08A
:1034900090FF0CC01F928F938EE997E09F938F93BC
:1034A0000E948A060F900F900F900F908091A502B6
:1034B0000F900F900F900F900F90DF91CF911F9171
:1034C0000F91FF90EF90DF90CF90BF900C941C264F
:1034D0000F900F900F900F900F90DF91CF911F9151
:1034E0000F91FF90EF90DF90CF90BF9008950C94D4
:1034F000290C0895EF92FF920F931F93CF93DF93C0
:1035000084EB97E00E94F105C0E0D0E08DE1E82E69
:1035100081E0F82E09EA17E08C2F0E941B0C0E9414
:10352000F825FF92EF921F928F93DF93CF931F9313
:103530000F930E948A0621968DB79EB708960FB604
:10354000F8949EBF0FBE8DBFC031D10529F7DF9122
:10355000CF911F910F91FF90EF90089508950895D6
:10356000CF93DF93CDB7DEB72B970FB6F894DEBFBE
:103570000FBECDBF942F4F83252F588769877A8739
:103580008B874A855B85452B31F02F3F31F481E0F5
:103590009F3F19F403C081E001C080E080FD07C0B7
:1035A0004F81588569857A858B850E940B26DE01BF
:1035B000119686E0FD0111928A95E9F785E0FE01FA
:1035C000379601900D928A95E1F749815A816B8176
:1035D0007C818D819E810E9406222B960FB6F894E5
:1035E000DEBF0FBECDBFDF91CF910895CF9388236B
:1035F00009F4C4C0C82F8CEF8C0F813A48F48C2F8B
:103600000E9444288111BAC08C2F0E94EE240CC065
:1036100080E28C0F883058F4C77081E001C0880FB9
:10362000CA95EAF70E949325CF910C94CD258BE59E
:103630008C0F833078F4C53A29F0C63A31F083E82C
:1036400090E005C081E890E002C082E890E0CF9170
:103650000C94761988E58C0F873108F08FC0C83A32
:1036600009F445C0C93A09F445C0CA3A09F445C04D
:10367000CB3A09F445C0CC3A09F445C0CD3A09F437
:1036800045C0CE3A09F445C0CF3A09F445C0C13B24
:1036900009F445C0C03B09F445C0C23B09F445C02C
:1036A000C33B09F445C0C43B09F445C0C53B09F41C
:1036B00045C0C63B09F445C0C73B09F445C0C83BFB
:1036C00009F445C0C93B09F445C0CA3B09F445C0EB
:1036D000CB3B09F445C0CC3B09F445C0CD3B09F4D4
:1036E00045C0CE3B09F445C080E090E044C082EE86
:1036F00090E041C089EE90E03EC08AEE90E03BC091
:1037000085EB90E038C086EB90E035C083EB90E02D
:1037100032C084EB90E02FC087EB90E02CC08CECA3
:1037200090E029C08DEC90E026C083E891E023C0B2
:103730008AE891E020C082E991E01DC084E991E02F
:103740001AC081E292E017C083E292E014C084E2E2
:1037500092E011C085E292E00EC086E292E00BC0DA
:1037600087E292E008C08AE292E005C08FE690E02E
:1037700002C080E790E0CF910C94A319CF910895F7
:10378000882329F19CEF980F913A18F40E943E2566
:103790000DC090E2980F983058F4877091E001C006
:1037A000990F8A95EAF7892F0E9499250C94CD25C7
:1037B0009BE5980F933020F480E090E00C9476190C
:1037C000885A873120F480E090E00C94A319089582
:1037D000882321F00E9493250C94CD2508958823F9
:1037E00021F00E9499250C94CD2508950E94B325BF
:1037F0000E9482250E94CD2580E090E00E947619EB
:1038000080E090E00C94A3190E94A3250C94F61B71
:10381000CF92DF92EF92FF920F931F93CF93DF939C
:1038200000D000D01F92CDB7DEB76C010E941E26DB
:10383000811101C385E0F601DE01119601900D9220
:103840008A95E1F7F6014081518123813481211568
:10385000310531F05F3F31F481E04F3F19F403C08F
:1038600081E001C080E080FDE6C2F601F280E580E3
:10387000E2948FE0E82249835A83FB82722F3D83D2
:103880002C836F2D8D810E946A248C010E946924F3
:103890000E945923E12FE295EF708E2F90E0FC01FA
:1038A000E15CFE4F0C949728812F807F1F70882346
:1038B00011F01295107FFF20B9F0112329F0812F0C
:1038C0000E94A6250E94CD25802F0F900F900F906B
:1038D0000F900F90DF91CF911F910F91FF90EF907C
:1038E000DF90CF900C94F61A802F0E94C01B1123FA
:1038F00009F4A1C2812F0E94AC250F900F900F9068
:103900000F900F90DF91CF911F910F91FF90EF904B
:10391000DF90CF900C94CD25812F807F1F70803257
:1039200011F01295107F002319F0013009F12BC01E
:10393000FF20A9F0EE2059F1F1E0812FEF1228C00D
:103940000F900F900F900F900F90DF91CF911F91DC
:103950000F91FF90EF90DF90CF900C94B625EE2062
:1039600021F021E0E21609F466C20E94B9254DC09B
:10397000FF20E9F085E08E1508F45DC20E949025D5
:10398000812329F042C0FF20F1F1E11015C0812F01
:103990000F900F900F900F900F90DF91CF911F918C
:1039A0000F91FF90EF90DF90CF900C94E81B94E084
:1039B0009E1508F440C229C0F601858180FF13C01E
:1039C0008F708583E4CF003F09F472C108F03EC1D7
:1039D00080E4800F803208F442C1FF2009F4D3C193
:1039E000EE2009F483C1802F0E94F61A093309F0F2
:1039F000C3C1FFEF21EE84E0F15020408040E1F7A9
:103A000000C0000018C2E110C0C1812F42C1812F47
:103A100086958695837019F08130B9F00CC2FF202D
:103A200019F0C801937002C080E090E00F900F90F1
:103A30000F900F900F90DF91CF911F910F91FF90FA
:103A4000EF90DF90CF900C947619FF2019F0C80109
:103A5000937002C080E090E00F900F900F900F9055
:103A60000F90DF91CF911F910F91FF90EF90DF901A
:103A7000CF900C94A319812F837009F070C0F110BE
:103A8000DAC1202F229526952770220F220F602F52
:103A90006F70862F90E0A0E0B0E06C017D01022EF7
:103AA00004C0CC0CDD1CEE1CFF1C0A94D2F704FFF2
:103AB00012C08FE090E0A0E0B0E004C0880F991F32
:103AC000AA1FBB1F2A95D2F7BC01CD016095709546
:103AD0008095909503C060E070E0CB011695169537
:103AE00013701230B1F040F56C297D298E299F2981
:103AF000113031F10F900F900F900F900F90DF91D8
:103B0000CF911F910F91FF90EF90DF90CF900C9489
:103B10007E236C297D298E299F290F900F900F906D
:103B20000F900F90DF91CF911F910F91FF90EF9029
:103B3000DF90CF900C9498230E947E23C701B6019A
:103B40000F900F900F900F900F90DF91CF911F91DA
:103B50000F91FF90EF90DF90CF900C946423FF20A3
:103B600019F0812F817001C08695882309F463C103
:103B7000202F229526952770220F220F602F6F701D
:103B8000862F90E0A0E0B0E06C017D01022E04C021
:103B9000CC0CDD1CEE1CFF1C0A94D2F704FF12C0F3
:103BA0008FE090E0A0E0B0E004C0880F991FAA1F4A
:103BB000BB1F2A95D2F7BC01CD0160957095809509
:103BC000909503C060E070E0CB01169516951370D8
:103BD0001230B1F040F56C297D298E299F291130D2
:103BE00031F10F900F900F900F900F90DF91CF91C8
:103BF0001F910F91FF90EF90DF90CF900C94452490
:103C00006C297D298E299F290F900F900F900F907E
:103C10000F90DF91CF911F910F91FF90EF90DF9068
:103C2000CF900C9457240E944524C701B6010F90F1
:103C30000F900F900F900F90DF91CF911F910F91E8
:103C4000FF90EF90DF90CF900C943324023F09F463
:103C50005EC008F449C0033F09F46CC0BECE902F8B
:103C60009071E92E812F8F71FF2051F00E94CC239B
:103C7000802FEE2019F08295807F8ACE8F7088CEBB
:103C80000E94ED23802FEE2019F08295807F01C0E5
:103C90008F700F900F900F900F900F90DF91CF913A
:103CA0001F910F91FF90EF90DF90CF900C94EF1B3E
:103CB000FF20A9F0E4E0EE1508F4BDC0812F8F715C
:103CC0000F900F900F900F900F90DF91CF911F9159
:103CD0000F91FF90EF90DF90CF900C941224F5E0BD
:103CE000FE1508F4A8C0EACFFF2099F0812F8F714C
:103CF0000F900F900F900F900F90DF91CF911F9129
:103D00000F91FF90EF90DF90CF900C94CC23FF2089
:103D100069F3812F8F710F900F900F900F900F907C
:103D2000DF91CF911F910F91FF90EF90DF90CF9097
:103D30000C94ED23FF2089F0812F8F710F900F904D
:103D40000F900F900F90DF91CF911F910F91FF90E7
:103D5000EF90DF90CF900C94B7230F900F900F90BF
:103D60000F900F90DF91CF911F910F91FF90EF90E7
:103D7000DF90CF900C94B223033509F43ACE073488
:103D800009F059C036CEEE2021F2802F0F900F900F
:103D90000F900F900F90DF91CF911F910F91FF9097
:103DA000EF90DF90CF900C94C01B412F4F70602F8D
:103DB000C6010E94DF260F900F900F900F900F907A
:103DC000DF91CF911F910F91FF90EF90DF90CF90F7
:103DD0000C94B42201112FC0FF2069F10E94041C31
:103DE0002FEF80E792E0215080409040E1F700C043
:103DF00000000F900F900F900F900F90DF91CF91D8
:103E00001F910F91FF90EF90DF90CF900C94C02600
:103E1000412F4F70602FC6010F900F900F900F90A1
:103E20000F90DF91CF911F910F91FF90EF90DF9056
:103E3000CF900C94E2260F900F900F900F900F9060
:103E4000DF91CF911F910F91FF90EF90DF90CF9076
:103E500008951F93CF93DF9300D000D01F92CDB76A
:103E6000DEB7942F4983252F5A836B837C838D8300
:103E70004C815D81452B31F02F3F31F481E09F3F34
:103E800019F403C081E001C080E0182F117080FD9B
:103E900024C049815A816B817C818D810E946A2472
:103EA000292F22952F702C3030F42A3048F42250DC
:103EB000223068F013C02C3061F02F3051F00EC06A
:103EC000803C28F0803E50F0815F833038F011E074
:103ED00005C093FB112710F901C010E0812F0F904E
:103EE0000F900F900F900F90DF91CF911F91089539
:103EF000CF93DF9300D000D01F92CDB7DEB70F90E5
:103F00000F900F900F900F90DF91CF910895CF9366
:103F1000DF9300D000D000D0CDB7DEB726960FB625
:103F2000F894DEBF0FBECDBFDF91CF9108951F93F0
:103F3000CF93DF93C091B60216E08091B702C81705
:103F400099F0D0E01C9FF0011D9FF00D1124E85462
:103F5000FD4F4081518162817381848195810E94EE
:103F6000871F2196C770E9CFDF91CF911F910895E8
:103F70004091E8025091E9026091EA027091EB02EF
:103F80008091EC029091ED020C94871F0F931F9388
:103F9000CF93DF938091ED0282958F7009F05DC021
:103FA0008091EA02882309F458C08091B6021091EA
:103FB000B7026091E8027091E902C091EB02D091E2
:103FC000EC0291E06F3F09F090E0292F06E08117A5
:103FD00009F443C0209721F07F3F21F030E003C077
:103FE00031E001C0322F90E030FD34C0089FF00175
:103FF000099FF00D1124DF01A854BD4F11963C918B
:104000001197371327C03C91361324C012963C9168
:10401000129731111FC013964D915C9114974C1B50
:104020005D0B483C5105B0F48091ED028F708061CA
:104030008093ED02E354FD4F80818F708061808317
:1040400088EE92E00E94081CDF91CF911F910F91A2
:104050000C94971F01968770BACFDF91CF911F9173
:104060000F9108959F92AF92BF92CF92DF92EF92FD
:10407000FF920F931F93CF93DF93CDB7DEB7619776
:104080000FB6F894DEBF0FBECDBF8C0185E0F801FE
:10409000DE011D9601900D928A95E1F7F8014081AD
:1040A0005181F280C380D4809091E8026091E9024E
:1040B0002091EB023091EC022115310531F06F3F78
:1040C00031F481E09F3F19F403C081E001C080E03A
:1040D000F82FF1709F2E80FD52C188EEA82E82E04D
:1040E000B82EE090EA02F601E21BF30BEE2009F491
:1040F000E8C08091ED02E83CF10508F0A4C0282F4B
:10410000207F09F053C0561313C0491311C0EF2C80
:10411000F1100EC08F7080618093ED020E94B81F75
:10412000C5010E94081C8091ED02F80185835BC1E6
:10413000C114D10431F05F3F31F481E04F3F19F4F5
:1041400003C081E001C080E080FD03C081E08F25D5
:1041500002C080E090E0F82FF170EF2E80FF1CC0CD
:104160008091B6022091B70236E0821709F418C197
:1041700090E0389FF001399FF00D1124E854FD4F75
:104180006181561306C06081461303C06281F61236
:1041900003C001968770E9CFEF2CFF2009F423C1FB
:1041A0008091ED0281608093ED0262C0561306C0DB
:1041B000491304C0F11002C0F801A7C04D875E8703
:1041C000FF867C2DD98AC88A6F2D89890E94291F74
:1041D000882399F1FF2089F12091ED02822F8295A9
:1041E0008F7090E0029774F08091E8029091E9025C
:1041F00098878F831986DB86CA862C87CE0107961F
:104200000E94081C86E0F801A8EEB2E001900D9231
:104210008A95E1F70E94C61F0E94B81F11C0561769
:1042200049F14D875E87FF867C2DD98AC88A6F2D1C
:1042300089890E94291F81112CC0C8010E94081C75
:10424000EE24E394D0C0282F207F49F77C2DD98A13
:10425000C88A6F2D89890E94781F88EE92E00E949B
:10426000081C86E0F50111928A95E9F70E94B81FB3
:10427000E12CB9C04913D5CFF110D3CFF801858314
:10428000C8010E94081C86E0F50111928A95E9F7A1
:10429000AAC0FF2091F22091ED02822F82958F70AB
:1042A00090E002970CF4AECF8091E8029091E90281
:1042B0009A8389831B82DD82CC822E83CE01019674
:1042C0009FCFE83CF10508F04BC0EF2CFF2009F42C
:1042D000B4CF561330C049132EC02091ED0220FDFB
:1042E00021C0822F82958F70482F50E041155105D3
:1042F000C9F0F80125834F30510541F08F5F982FA9
:104300009295907F822F8F70892B8583C8010E94A0
:10431000081C86E0F801A8EEB2E001900D928A95A3
:10432000E1F72AC086E0F801A8EEB2E001900D9214
:104330008A95E1F758C04D875E87FF867C2DD98A24
:10434000C88A6F2D89890E94291F81115BCF8091B6
:10435000ED0281608093ED02C8010E94081C43C0F9
:104360007C2DD98AC88A6F2D89890E94781F86E0A2
:10437000F50111928A95E9F70E94B81F34C0FF2019
:1043800009F45BCF4D875E87FF867C2DD98AC88A6A
:104390006F2D89890E94291F882309F44ECF32CFBF
:1043A0007C2DD98AC88A6F2D89890E946A24292F79
:1043B00022952F70223028F49F7039F0811105C0AA
:1043C0000BC0243028F49F7049F4805E883020F0C0
:1043D000C8010E94081C9E2CE92C05C0F80195819B
:1043E000907F99F7F9CF8E2D61960FB6F894DEBFC6
:1043F0000FBECDBFDF91CF911F910F91FF90EF9036
:10440000DF90CF90BF90AF909F9008951F93CF9370
:10441000DF93CDB7DEB72C970FB6F894DEBF0FBE93
:10442000CDBF4F83588769877A878B879C87CE015A
:1044300007960E9432208823D1F09F8188852A85A3
:104440003B85232B31F08F3F31F481E09F3F19F4FE
:1044500003C081E001C080E080FD47C04F815885E6
:1044600069857A858B859C850E94871F3EC086E082
:10447000FE013796DE01119601900D928A95E1F7C3
:10448000FF81E8856A857B856115710531F0EF3F15
:1044900031F481E0FF3F19F403C081E001C080E006
:1044A00080FD23C02091B70230E0C90101968770DA
:1044B00099274091B60250E084179507F1F1F983EE
:1044C000EA837D836C8396E0929FD001939FB00D29
:1044D0001124A854BD4FFE01319601900D929A957A
:1044E000E1F78093B7020E94971F16E08091B60211
:1044F0009091B702891771F1189FC0011124885457
:104500009D4F0E943220882329F1E091B6021E9F20
:10451000F0011124E854FD4F408151816281738183
:10452000848195810E94871F8091B60290E0019658
:10453000877099278093B602D9CF0E94041C1092ED
:10454000B7021092B602E8EEF2E086E0DF011D92BB
:104550008A95E9F72C960FB6F894DEBF0FBECDBF53
:10456000DF91CF911F910895DF92EF92FF920F9309
:104570001F93CF93DF93FC01892B09F488C0E12CB2
:10458000F12CDD24D394EF0121968491853709F431
:1045900060C058F4843708F04EC0843008F068C01A
:1045A0008130D1F0823071F172C0883709F45BC07C
:1045B00050F4863709F453C0873709F068C08E2D50
:1045C0000E94A02552C09CE7980F903708F05FC06A
:1045D0008F770E94C01B4EC08F010E5F1F4FFE01E0
:1045E000849190E2980F983050F48770FD2D01C0AF
:1045F000FF0F8A95EAF78F2F0E94A62515C00E940B
:10460000F61A14C08F010E5F1F4FFE01849190E2D5
:10461000980F983068F48770FD2D01C0FF0F8A95C0
:10462000EAF78F2F0E94AC250E94CD25E80122C019
:104630000E94C01BFBCFCF010296FE01C491CC2388
:1046400061F0EFE9FFE03197F1F700C00000C150E1
:10465000F6CFCF010296FE01F490EC010BC00E9450
:104660009025E82E07C00E94A3250E94CD2502C0F8
:104670000E94F61A8F2D882341F0EFE9FFE0319771
:10468000F1F700C000008150F6CFFE017CCFDF9132
:10469000CF911F910F91FF90EF90DF90089560935D
:1046A0006E0370936F0380937003909371030C9467
:1046B0001B260895609372037093730380937403B1
:1046C000909375030C941A260F931F930091720315
:1046D000109173032091740330917503602B712B3B
:1046E000822B932B609372037093730380937403F4
:1046F000909375031F910F910C941A260F931F939B
:10470000009172031091730320917403309175032B
:104710006023712382239323609372037093730346
:1047200080937403909375031F910F910C941A2634
:104730000F931F93009172031091730320917403E0
:104740003091750360277127822793276093720346
:104750007093730380937403909375031F910F916B
:104760000C941A2660E070E0CB010C944F230F9359
:104770001F9341E050E060E070E08A019B0104C0BB
:10478000000F111F221F331F8A95D2F7C901B801EC
:104790001F910F910C944F230F931F9341E050E012
:1047A00060E070E004C0440F551F661F771F8A95B4
:1047B000D2F780916E0390916F03A0917003B09136
:1047C00071038A019B01082B192B2A2B3B2BC90152
:1047D000B8011F910F910C944F230F931F9341E049
:1047E00050E060E070E004C0440F551F661F771F63
:1047F0008A95D2F7409550956095709580916E039B
:1048000090916F03A0917003B09171038A019B0195
:10481000082319232A233B23C901B8011F910F91B3
:104820000C944F230F931F9341E050E060E070E041
:1048300004C0440F551F661F771F8A95D2F78091D9
:104840006E0390916F03A0917003B09171038A0180
:104850009B01082719272A273B27C901B8011F9167
:104860000F910C944F230F931F9300916E0310919F
:104870006F032091700330917103602B712B822B99
:10488000932B1F910F910C944F230F931F93009123
:104890006E0310916F0320917003309171036023B8
:1048A0007123822393231F910F910C944F230F9315
:1048B0001F9300916E0310916F032091700330914C
:1048C000710360277127822793271F910F910C9402
:1048D0004F2308958F929F92AF92BF92DF92EF92F3
:1048E000FF920F931F93CF93DF9300D000D01F92BE
:1048F000CDB7DEB76B837C838D838A018C819D81EC
:10490000892B31F01F3F31F481E04F3F19F403C090
:1049100081E001C080E080FF03C080E090E04DC0F6
:104920008B818823D1F180906E0390906F03A090CB
:104930007003B09071038091720390917303A09102
:104940007403B0917503882A992AAA2ABB2A8FE199
:10495000E82EF12CD501C4010E2C04C0B695A79504
:10496000979587950A94D2F780FD06C081E0E81AF2
:10497000F10880F7D12C07C0DE2CB8018E2D0E94E3
:104980009306019799F388E0189FF0011124E251F2
:10499000FD4FE00FF11DD08209C088E0189FF001A3
:1049A0001124E251FD4FE00FF11DD08009831A83DD
:1049B00069817A818D2D0E9493060F900F900F9040
:1049C0000F900F90DF91CF911F910F91FF90EF907B
:1049D000DF90BF90AF909F908F90089590911401B9
:1049E000992379F190911501992359F1982F969572
:1049F000969596959F31A1F0E0911601F0911701DF
:104A0000E90FF11D877021E030E0A90102C0440FD9
:104A1000551F8A95E2F7CA019181892B81830895F8
:104A20009091990390FF29C01F928F938FED97E08B
:104A30009F938F930E948A060F900F900F900F9074
:104A400008952091160130911701F90132969FEFD8
:104A500040E05191851789F09F3F19F4511101C031
:104A6000942F4F5F4E31A9F79F3F39F0F901E90FBD
:104A7000F11D97FDFA958283089508959091140190
:104A8000992381F190911501992361F1982F9695C1
:104A9000969596959F31A9F0E0911601F091170136
:104AA000E90FF11D877021E030E0A90102C0440F39
:104AB000551F8A95E2F7CA018095918189238183E8
:104AC00008959091990390FF1CC01F928F9381ECE1
:104AD00097E09F938F930E948A060F900F900F90FC
:104AE0000F900895E0911601F09117019F01225E49
:104AF0003F4F9281891301C012823196E217F3076A
:104B0000C1F7089581E090E0E0911601F09117015E
:104B1000E80FF91F1082019680329105A9F70895D8
:104B200080919803089590919803892B809398031E
:104B30000895809590919803892380939803089510
:104B40008093980308951092980308959091970385
:104B5000892B8093970308958095909197038923DB
:104B60008093970308951092970308958093760396
:104B7000089510927603089580911601909117017F
:104B8000FC0131969C01205E3F4F80E09191911194
:104B90008F5FE217F307D1F70895E0911601F091C6
:104BA0001701809198038083E0911601F09117011D
:104BB000908180919703892B80838091760388234D
:104BC00061F0E0911601F09117019081892B8083AB
:104BD0000E94BC258111109276038091160190915C
:104BE00017010C942D199093590180935801089541
:104BF0008295982F937344E0949F900111248C7CAC
:104C000086958695282B822F8575880F2A7A26957A
:104C1000822B08950895CF93DF9300D000D01F9288
:104C2000CDB7DEB70F900F900F900F900F90DF91E0
:104C3000CF910895089508950C94771A80E008950F
:104C400083B7817F8C6083BF83B7816083BF789493
:104C5000889583B78E7F83BF0895CF930E94AE1A45
:104C60000E94380C0E94AF1AC0E08C2F0E941B0CCF
:104C7000811104C0CF5FC031C1F701C081E0CF9185
:104C800008950E94210C0C94041C1F920F920FB6E1
:104C90000F9211248F939F93AF93BF9380919A03A8
:104CA00090919B03A0919C03B0919D034196A11DFF
:104CB000B11D80939A0390939B03A0939C03B093A0
:104CC0009D03BF91AF919F918F910F900FBE0F9059
:104CD0001F90189582E084BD93E095BD9AEF97BD33
:104CE00080936E0008952FB7F89480919A03909165
:104CF0009B03A0919C03B0919D032FBF08952FB7F4
:104D0000F89460919A0370919B0380919C03909119
:104D10009D032FBF08959C014FB7F89480919A038B
:104D200090919B03A0919C03B0919D034FBF821B68
:104D3000930B089578941F920F920FB60F9211243F
:104D40008F939F93AF93BF9380919A0390919B030E
:104D5000A0919C03B0919D030196A11DB11D80936C
:104D60009A0390939B03A0939C03B0939D03BF91E0
:104D7000AF919F918F910F900FBE0F901F9018953C
:104D80000E94B117F89487E797E790930108809302
:104D9000000887E090EBDC018093AC039093AD03B7
:104DA000A093AE03B093AF039CE088E10FB6F894F4
:104DB000A895809360000FBE90936000FFCF80E0C5
:104DC00090E008950895CF93C82F1F928F9383E0AA
:104DD00098E09F938F930E948A0681E090E0A0E084
:104DE000B0E0BC01CD0104C0660F771F881F991F7A
:104DF000CA95D2F70E945A230F900F900F900F90F0
:104E0000CF910C94041CCF938732A8F58E3108F013
:104E10002BC1803109F49FC0F8F4873009F464C0D5
:104E2000A8F4863009F024C180919903817F8E7F98
:104E30008093990388E098E00E94F1058BEE9AE058
:104E40000E94F10581E080939E034CC08B30F1F10C
:104E50008E3009F46CC00CC1863109F4B0C020F466
:104E6000813109F4EDC004C1893109F491C08B315D
:104E700009F449C0FDC0883349F150F4893209F47E
:104E8000F1C0853309F4EEC0873209F0F1C0EAC001
:104E9000833409F4E7C028F48A3308F4E9C089535D
:104EA000E4C0883409F0E4C00E94041C8AED9AE052
:104EB0000E94F1052FEF83ED90E321508040904058
:104EC000E1F700C000000E94C0260CC083E298E019
:104ED0005CC081EC9AE00E94F105809199038160A9
:104EE00080939903C1E0C9C080919903C82FC17014
:104EF00080FFEFCF8DEC9AE00E94F105809199033D
:104F0000817F8E7F3DC09091990391FBCC27C0F9A2
:104F100081E0C827892FC0FB81F980939903CC23B6
:104F200019F084EB9AE027C086EA9AE02EC09091AF
:104F3000990392FBCC27C0F981E0C827892FC0FBD9
:104F400082F980939903CC2319F087E99AE013C082
:104F500087E89AE01AC09091990393FBCC27C0F997
:104F600081E0C827892FC0FB83F980939903CC2364
:104F700051F08BE79AE00E94F105809199038160DE
:104F8000809399037AC08EE69AE00E94F105AACF39
:104F90008FE59AE00E94F10589E39AE00E94F1050D
:104FA00081EF99E00E94F10589EC99E00E94F105FA
:104FB0008DE799E00E94F10581E599E0E6CF83E471
:104FC00099E00E94F1050E9421191F928F9389E2B6
:104FD00099E09F938F930E948A06809114011F92FB
:104FE0008F9382E199E09F938F930E948A0680912C
:104FF0009E021F928F938FEF98E09F938F930E9452
:105000008A06809115011F928F938CEE98E09F93F2
:105010008F930E948A060E947F269F938F937F938F
:105020006F9385ED98E09F938F930E948A068DB7CA
:105030009EB746960FB6F8949EBF0FBE8DBF52CF57
:105040000E94041CC091150181E0C827C09315017E
:10505000CC2329F08BEC98E00E94F1050EC080EC87
:1050600098E093CF80E001C08D510E94E3263ACFB3
:105070008EEB98E00E94F105C0E08C2FCF9108954F
:1050800080E008950C944028CF93C82F80919E0310
:10509000882319F0813059F042C0E0911601F09157
:1050A00017018081823261F08434D9F509C0E09122
:1050B0001601F09117018081823211F0843461F47D
:1050C0008C2F0E944228811104C08C2F0E9403273C
:1050D00024C081E090E021C08C2F0E9440288111E3
:1050E0001BC0C43189F018F4CB3029F010C0C9328C
:1050F00059F0C83361F488E098E00E94F1058FEF21
:1051000097E00E94F10508C010929E030CC08DEF3D
:1051100097E00E94F10507C081E0817006C01092FF
:105120009E0380E002C080E0F8CFCF910895EE0F9B
:10513000FF1F0024001C0BBE0790F691E02D099480
:04514000F894FFCF11
:105144000080FFFF057D010000FFD9104611DC102F
:105154001111DD10010177035F5A313530005F3FD3
:105164003F3F3F005F4154383400415400585400DD
:105174004E4F4E45005445524D494E414C00403629
:1051840022392D07F706D5069C06280641065A063D
:085194007A0600100008000477
:106800008800EA44E944E244040005000600070069
:10681000080009000A000B000C000D000E000F001C
:1068200010001100120013001400150016001700CC
:10683000180019001A001B001C001D001E001F007C
:10684000200021002200230024002500260027002C
:10685000280029002A002B002C002D002E002F00DC
:10686000300031003200330034003500360037008C
:10687000380039003A003B003C003D003E003F003C
:1068800040004100420043004400450046004700EC
:10689000480049004A004B004C004D004E004F009C
:1068A000500051005200530054005500560057004C
:1068B000580059005A005B005C005D005E005F00FC
:1068C0006000610062006300640065A185006700EC
:1068D000680069006A006B006C006D006E006F005C
:1068E0007000710072007300890087008A008B00BD
:1068F000E000E100E200E300E400E500E600E7007C
:106900000100010001000100EA4401000100E2442D
:106910000100010001000100460001004A004B0097
:10692000010001004700480001000100E9440100A6
:106930000100010001000100010001003A003B00DC
:106940003C003D003E003F0040004100420043004B
:10695000010035004C0039000100440045005200A0
:1069600049000100010050004F0029004D004E0079
:1069700051000100010001000100010001000100BF
:1069800001000100010001000100010001000100FF
:1069900001000100010001000100010001004D00A3
:1069A0004A004E004B0001000100010001000100FF
:1069B00001000100010001000100010001000100CF
:1069C00001000100010001000100010001000100BF
:1069D00001000100010001000100010001000100AF
:1069E0000100010001000100490001000100010057
:1069F000010001000100010001000100010001008F
:00000001FF
